:100000000C9470010C948D010C948D010C948D0155
:100010000C948D010C948D010C948D010C948D0128
:100020000C948D010C948D010C94E91D0C94BB1E55
:100030000C94F0180C948D010C948D010C948D018E
:100040000C948D010C948D010C948D010C948D01F8
:100050000C948D010C9478190C948D010C948D01E5
:100060000C948D010C948D010C948D010C948D01D8
:100070000C948D010C948D010C948D010C948D01C8
:100080000C948D010C948D010C948D010C948D01B8
:100090000C948D010C948D010C948D010C948D01A8
:1000A0000C948D010C948D010C948D01B104B1045C
:1000B000DD04DD04450563057B067B066E0507064A
:1000C00018061806281F4F1F47204F1F47209B1F49
:1000D000BE1F472015202420530054005500560011
:1000E0005F00600061002B005C005D005E00570057
:1000F00059005A005B004C006200A75D6300580085
:1001000000000000000000002A2B28000000000072
:1001100000000000000000000000002900000000B6
:100120002C1E3420212224342627252E362D373824
:10013000271E1F202122232425263333362E37382D
:100140001F0405060708090A0B0C0D0E0F101112EB
:10015000131415161718191A1B1C1D2F3130232DB7
:10016000350405060708090A0B0C0D0E0F101112B5
:10017000131415161718191A1B1C1D2F3130354C66
:10018000000000000000000000000000000000006F
:10019000000000000000000000000000000000005F
:1001A000000000007E0F00D4FFFFFFC700000078B2
:1001B000120350003200300020007600650072000B
:1001C000320000000E0350006100620069006C0004
:1001D000650000000403090409023B00020100A0BD
:1001E000FA090400000103010100092111010001C5
:1001F00022400007058103080001090401000103F2
:10020000000000092111010001227B000705820383
:100210002000011201000200000008666667660205
:10022000000102000105010902A10185020901A1E5
:100230000005091901290815002501950875018196
:10024000020501093009311581257F950275088164
:100250000609381581257F950175088106050C0A68
:1002600038021581257F950175088106C0C00501FA
:100270000980A101850319012AB700150126B700DD
:10028000950175108100C0050C0901A101850419B3
:10029000012AA002150126A002950175108100C057
:1002A00005010906A101050719E029E71500250147
:1002B00095087501810295017508810105071900EE
:1002C00029FF150026FF009506750881000508190D
:1002D000012905950575019102950175039101C0EC
:1002E00011241FBECFEFDAE0DEBFCDBF11E0A0E0EA
:1002F000B1E0E4EFF1E402C005900D92A438B1073B
:10030000D9F722E0A4E8B1E001C01D92A634B207FB
:10031000E1F70E944D120C94F8200C940000873AEB
:100320009D4551F4FB018281882331F082E60E94D1
:100330005F0482E60E945F0481E008959C013A9583
:1003400021153F4130F5BC0166277270AC0144278E
:1003500054709C012227387094FF0FC090FF02C098
:1003600080E101C080E0672B09F08062452B09F035
:100370008064232B79F080680895892F8170672B22
:1003800009F08260452B09F08460232B19F0886006
:10039000089580E00895CF93DF93EB010E949E01C2
:1003A000FE01DF91CF910994CF93DF93EC01805E42
:1003B0009109089710F0209719F468E674E002C0DC
:1003C00063EF76E0CE010E94CB018C2FDF91CF91BD
:1003D0000C94BE03CF93DF93EC010E941404CE0172
:1003E000805E9109089710F0209719F46FE674E089
:1003F00002C06AEF76E0CE01DF91CF910C94CB0181
:10040000CF93DF93EC010E94D401C933D10549F4A5
:100410002FEF87EE93E0215080409040E1F700C03D
:100420000000CE01DF91CF910C94EA0181E00895A4
:100430000C948F0108950C941A021F93CF93DF93AD
:1004400000D000D01F92CDB7DEB749835A836B83AB
:100450003091870189819A81311114C0662359F046
:10046000222349F00E94C408182F682F89819A819D
:100470000E946F0803C00E949908182F69817A8131
:10048000812F04C00E94C40869817A810F900F9067
:100490000F900F900F90DF91CF911F910C94E40F6C
:1004A000FC01262F408151816281738184810C94EB
:1004B0001D0281E00895CF93DF93EC0160E00E947C
:1004C0005002BE01DF91CF910C941B020C941111CC
:1004D0000C940D1108950E9419070E946A022FEFD3
:1004E00084E39CE0215080409040E1F700C0000090
:1004F0000C949E190F931F93CF93DF938C0161E0AF
:100500000E945002EC01B8010E941802882309F4ED
:1005100044C0B801CE010E94AF158823F1F1B801A3
:10052000CE010E94B9178823C1F1B801CE010E9403
:10053000CD15882391F1B801CE010E9415178823AB
:1005400061F1F8018281882309F1CB358DE5D80767
:10055000C1F050F4C115FCE5DF0781F0CF3DDC456B
:10056000A9F40E94F80D19C0CC35EDE5DE0761F065
:10057000CD35DD4559F40E94410D08C00E946B0243
:100580000CC00E944A0D02C00E944D0DC801DF91AF
:10059000CF911F910F910C94160280E0DF91CF91C3
:1005A0001F910F9108950E94D3180C945C030E9430
:1005B0005F030C94D918DF92EF92FF920F931F9371
:1005C000CF93DF93E82FF0E0E050FF4FD490282F37
:1005D00026952695269530E0F901E056FE4F0491C8
:1005E000877010E0082E02C0159507950A94E2F76F
:1005F00001701127F901E057FE4FE490F12C082E0D
:1006000002C0F594E7940A94E2F791E0E922FF240E
:10061000F901E058FE4FC491D0E002C0D595C795CE
:100620008A95E2F7C170DD270115110519F081EEF9
:100630000E94BE03E114F10419F086EE0E94BE038D
:100640008D2D0E945F04EF2819F086EE0E9414049D
:10065000012B19F081EE0E941404CD2B51F08CE295
:10066000DF91CF911F910F91FF90EF90DF900C944D
:100670005F04DF91CF911F910F91FF90EF90DF907A
:100680000895982F9F709A50963010F0805D01C0A9
:10069000895A0C94DB0208950C944B0381E0089571
:1006A0000C944E030895CF93C82F0E944C038C2FB7
:1006B0000E945003CF91089580E00C9453030E9450
:1006C00015180C9453030E941518909186018917F0
:1006D00021F0809386010C9453030895CF93DF9308
:1006E000CDB7DEB72B970FB6F894DEBF0FBECDBFE8
:1006F0004F83588769877A878B8761110E948D0C99
:100700009E012F5F3F4F86E0F90111928A95E9F72C
:1007100085E0FE013796D90101900D928A95E1F7A7
:1007200089819A814C815D81452B31F09F3F31F465
:1007300091E08F3F19F403C091E001C090E090FF79
:1007400009C049815A816B817C818D819E810E9483
:10075000AB0B05C0C9010E9459028111F2CF2B9643
:100760000FB6F894DEBF0FBECDBFDF91CF910895D5
:10077000FC01808191810E9406090895CF9388230E
:1007800009F450C0C82F8CEF8C0F813AD0F46C2F35
:1007900080910201909103010E947518882349F00D
:1007A0006C2F80910201909103010E94AD180E946C
:1007B000AF0C6C2F80910201909103010E94AB1845
:1007C0000CC080E28C0F883058F4C77081E001C003
:1007D000880FCA95EAF70E946D0CCF910C94AF0C6C
:1007E000EBE5EC0FE33040F4F0E0E95BFE4F808195
:1007F00090E0CF910C943D18E8E5EC0FE73150F410
:10080000F0E0EE0FFF1FE75EFE4F80819181CF91F8
:100810000C945318CD3E30F08C2F0E94D212CF9101
:100820000C94A413CF910895882389F19CEF980F1D
:10083000913A40F4682F80910201909103010E9447
:10084000AD180DC090E2980F983058F4877091E081
:1008500001C0990F8A95EAF7892F0E94730C0C94B6
:10086000AF0C9BE5980F933020F480E090E00C945F
:100870003D1898E5980F973120F480E090E00C94B3
:1008800053188D3E20F00E942D130C94A41308954C
:100890001F93CF93DF93182FEB010E94BE03209785
:1008A00041F08FE99FE00197F1F700C00000219728
:1008B000F6CF812FDF91CF911F910C9414048933CF
:1008C00019F060E070E002C060E570E00C9448044C
:1008D000882321F00E946D0C0C94AF0C089588239E
:1008E00021F00E94730C0C94AF0C0895CF92DF920C
:1008F000EF92FF920F931F93CF93DF937C01D62F3C
:10090000C72FFC011281058102950F700E94630CB4
:100910008823B9F01123A9F08C2F807F803421F037
:1009200080E28D0F883068F08091230282FD09C03B
:1009300082E00E940F0D0E94630C91E0D82ED92610
:1009400001C0D12CCC2EC2948FE0C8228C2D90E017
:100950008C30910508F0CFC1FC01EA5AFF4F0C948E
:100960008F208C2F807FCF70882311F0C295C07F9D
:10097000112399F0CC2309F4AAC180E28D0F8830AD
:1009800010F0D11104C08C2F0E946D0C03C08C2F6D
:100990000E94800C0E94AF0C9AC18D2F0E941404FB
:1009A000CC2309F4A8C180E28D0F883038F1DD2313
:1009B00029F18C2F0E94860C24C08C2F807FCF7051
:1009C000803211F0C295C07FDD2319F0D130A1F142
:1009D0003DC08091230282FF17C0112349F0CC2330
:1009E00029F08C2F0E946D0C0E94AF0C80E070C12A
:1009F00080E00E941404CC2309F47DC18C2F0E9456
:100A0000730C0E94AF0C77C1112371F0002341F0E9
:100A1000013031F40E94900C8C2B0E94980C6BC119
:100A20000E94900C8C2B1DC0002319F0013009F49A
:100A300062C10E94A50C25C0112321F0063008F0E8
:100A40005AC10EC0053008F056C11BC0112361F019
:100A5000002331F0F701858180FF39C18F708583D4
:100A60008C2F0E94680447C1002359F0D93309F044
:100A70003FC1FFEF07EE13E0F15000401040E1F7F7
:100A800035C18C2F0E946F0436C18C2F86958695B8
:100A9000837019F0813061F02EC1112321F08D2F68
:100AA0009C2F937002C080E090E00E943D182BC103
:100AB000112321F08D2F9C2F937002C080E090E0D5
:100AC0000E94531820C18D2F112319F00E94D212B9
:100AD00002C00E942D130E94A41315C18C2F837095
:100AE00009F047C011110BC12D2F229526952770B3
:100AF000220F220F6D2F6F70862F90E0A0E0B0E0E4
:100B0000022E04C0880F991FAA1FBB1F0A94D2F798
:100B1000D4FF10C04FE050E060E070E004C0440F2C
:100B2000551F661F771F2A95D2F7409550956095FF
:100B3000709503C040E050E0BA01C695C695C370F9
:100B40008A019B01082B192B2A2B3B2BC901B801C9
:100B5000C23049F058F4C13019F00E948507CFC067
:100B60000E947307CCC00E949707C9C00E947107FA
:100B7000C6C0112319F08C2F817001C0869588237F
:100B800009F4BDC02D2F229526952770220F220F24
:100B90006D2F6F70862F90E0A0E0B0E0022E04C0B1
:100BA000880F991FAA1FBB1F0A94D2F7D4FF10C049
:100BB0004FE050E060E070E004C0440F551F661F36
:100BC000771F2A95D2F7409550956095709503C090
:100BD00040E050E0BA01C695C695C3708A019B01FA
:100BE000082B192B2A2B3B2BC901B801C23049F025
:100BF00058F4C13019F00E944A0881C00E94380898
:100C00007EC00E945C087BC00E94AB0778C0CF709A
:100C1000112339F08C2F0E94D1078D2F0E94680478
:100C20006EC08D2F0E946F048C2F0E94F20767C048
:100C3000D23F21F128F4D03F41F0D13FC1F043C071
:100C4000D33F19F1D43F79F03EC0112341F0053074
:100C500008F051C08C2F8F710E9417084CC00630CD
:100C600008F049C0F7CF8091230282FF18C01123FA
:100C700039F08C2F8F710E94D1073DC01123C9F329
:100C80008C2F8F710E94F20736C0112329F08C2F10
:100C90008F710E94BC072FC00E94B7072CC0112380
:100CA00049F0CF718C2F0E94D10763E08C2F0E94F6
:100CB000F40C21C081E00E940F0D0230E0F082E0D0
:100CC0000E940F0D18C0112331F0002391F28D2FD7
:100CD0000E94BE0310C0002399F2D93349F41FEFDC
:100CE00027EE33E0115020403040E1F700C0000013
:100CF0008D2F0E94140488EF8C0D843020F40E9404
:100D000015180E945303DD20C9F00E945F0C80FD7E
:100D100015C0F70112820E94590C0E94D107C70129
:100D20000E94BF060E94590CDF91CF911F910F9135
:100D3000FF90EF90DF90CF900C94F207DF91CF916E
:100D40001F910F91FF90EF90DF90CF9008950F9338
:100D50001F93CF93DF93EC01688179818A810E9490
:100D600011098C010E946E080E945F07B801CE0134
:100D70000E947604DF91CF911F910F910895CF9338
:100D8000DF93EC01988189812B813C81232B31F009
:100D90008F3F31F481E09F3F19F403C081E001C02F
:100DA00080E080FD1DC0CE010E947A02811110C03A
:100DB0000E94630C8823A1F08A81882389F08091A6
:100DC000230282FD0DC082E0DF91CF910C940F0DC4
:100DD000CE010E94A706CE01DF91CF910C945B0259
:100DE000DF91CF910895882321F00E94800C0C940C
:100DF000AF0C0895882321F00E94860C0C94AF0C50
:100E0000089580E090E00E943D1880E090E00E940C
:100E100053180E948D0C0E94AF0C0E94D5140C94A4
:100E2000A41380910201909103010E94AF180C94C9
:100E300001070E947D0C0C94110792959F709630CB
:100E400079F010F4925001C09A50923068F4803FCB
:100E500069F018F4883E40F409C0843F29F406C0C4
:100E6000883E20F0813F11F080E0089581E00895F0
:100E7000FC01808191810E9406090E941D0708954E
:100E8000CF93DF9300D000D01F92CDB7DEB70F9085
:100E90000F900F900F900F90DF91CF910895CF9307
:100EA000DF9300D000D000D0CDB7DEB726960FB6C6
:100EB000F894DEBF0FBECDBFDF91CF9108950895A6
:100EC00008950C9460070C9461070E946307609377
:100ED0009B0170939C0180939D0190939E010C94C3
:100EE00001070C9465070F931F9300919B011091CC
:100EF0009C0120919D0130919E01602B712B822BD2
:100F0000932B1F910F910C9465070F931F930091E2
:100F10009B0110919C0120919D0130919E016023C5
:100F20007123822393231F910F910C9465070F93D4
:100F30001F9300919B0110919C0120919D01309184
:100F40009E0160277127822793271F910F910C9490
:100F500065070C9460070E94A9076093970170933E
:100F600098018093990190939A010C94010760E095
:100F700070E0CB010C94AB070F931F9341E050E05E
:100F800060E070E08A019B0104C0000F111F221F66
:100F9000331F8A95D2F7C901B8011F910F910C94A4
:100FA000AB070F931F9341E050E060E070E004C096
:100FB000440F551F661F771F8A95D2F780919701BE
:100FC00090919801A0919901B0919A018A019B0199
:100FD000082B192B2A2B3B2BC901B8011F910F910C
:100FE0000C94AB070F931F9341E050E060E070E07A
:100FF00004C0440F551F661F771F8A95D2F740958E
:101000005095609570958091970190919801A0916D
:101010009901B0919A018A019B01082319232A237F
:101020003B23C901B8011F910F910C94AB070F939B
:101030001F9341E050E060E070E004C0440F551F92
:10104000661F771F8A95D2F780919701909198013A
:10105000A0919901B0919A018A019B010827192753
:101060002A273B27C901B8011F910F910C94AB07A8
:101070000F931F930091970110919801209199016E
:1010800030919A01602B712B822B932B1F910F9122
:101090000C94AB070F931F93009197011091980147
:1010A0002091990130919A01602371238223932327
:1010B0001F910F910C94AB070F931F930091970111
:1010C000109198012091990130919A016027712720
:1010D000822793271F910F910C94AB070895990FC6
:1010E000990F890FE82FE695E695E695877051E010
:1010F00001C0550F8A95EAF785E0E89FF0011124B9
:10110000E857FE4F20E030E070E04081CB01022E36
:1011100002C0969587950A94E2F78170819584279D
:101120008523842781932F5F3F4F2530310569F751
:101130000895990F990F890F682F669566956695A2
:10114000982F977085E0689FB001112440E050E02F
:1011500080E0FB01E40FF51FE857FE4F208130E0EF
:10116000092E02C0369527950A94E2F7217033279D
:10117000042E01C0220F0A94EAF7822B4F5F5F4FC3
:101180004530510531F70895BF92CF92DF92EF922B
:10119000FF920F931F93CF93DF938C01C090970121
:1011A000D0909801E0909901F0909A0180919B0174
:1011B00090919C01A0919D01B0919E01C82AD92ACD
:1011C000EA2AFB2ACFE1D0E0D701C6010C2E04C0E9
:1011D000B695A795979587950A94D2F780FD04C098
:1011E000219790F7B12C07C0BC2EB8018C2F0E941C
:1011F000F80F0197A9F38B2DDF91CF911F910F91DC
:10120000FF90EF90DF90CF90BF900895CF93DF9342
:10121000EC010E94C408BE010E94F80FDF91CF913B
:1012200008951F93CF93DF93EB019091870199234A
:1012300021F0CB010E94060913C0882349F0CB019D
:101240000E94C408182F682FCE010E946F0804C0A6
:10125000CB010E949908182FBE01812F0E94F80F20
:10126000DF91CF911F9108951F93CF93DF93C0918A
:101270009F0116E08091A001C81799F0D0E01C9F53
:10128000F0011D9FF00D1124EF55FE4F408151815B
:1012900062817381848195810E944F072196C77076
:1012A000E9CFDF91CF911F9108954091D1015091E5
:1012B000D2016091D3017091D4018091D5019091B8
:1012C000D6010C944F07EF92FF920F931F93CF9389
:1012D000DF938091D60182958F7009F065C080916F
:1012E000D301882309F460C080919F01F090A00190
:1012F0001091D1010091D2016091D4017091D5017A
:1013000091E01F3F09F090E0C0910001D0910101F0
:10131000292F96E0E92E8F1509F446C06115710555
:1013200021F00F3F21F030E003C031E001C0322F47
:1013300090E030FD36C0E89EF001E99EF00D1124EA
:10134000DF01AF55BE4F11963C911197301329C064
:101350003C91311326C012963C911297311121C055
:1013600013964D915C911497461B570B4C175D07D4
:10137000C0F48091D6018F7080618093D601EA55C8
:10138000FE4F80818F708061808381ED91E00E94AB
:10139000BF06DF91CF911F910F91FF90EF900C94BA
:1013A000340901968770B7CFDF91CF911F910F91CC
:1013B000FF90EF9008959F92AF92BF92CF92DF92ED
:1013C000EF92FF920F931F93CF93DF93CDB7DEB7CA
:1013D00061970FB6F894DEBF0FBECDBF8C0185E0DC
:1013E000F801DE011D9601900D928A95E1F7D80172
:1013F0001296EC909091D101E091D2012091D4010C
:101400003091D5012115310531F0EF3F31F481E004
:101410009F3F19F403C081E001C080E0B82FB17094
:101420009B2E80FD47C1D8014C9111965C9111977C
:101430001396AD90BC90149781EDC82E81E0D82E04
:10144000F090D301B501621B730B20910001309124
:101450000101FF2009F4D9C08091D60162177307FA
:1014600008F095C0282F207F09F052C05E1313C0EA
:10147000491311C0FE2CE1100EC08F708061809363
:10148000D6010E945509C6010E94BF068091D6016F
:10149000F80185834DC1AB2831F05F3F31F481E025
:1014A0004F3F19F403C081E001C080E080FD03C01C
:1014B00081E08E2502C080E090E0F82FF170FF2ED1
:1014C00080FF1CC080919F012091A00136E082170F
:1014D00009F40BC190E0389FF001399FF00D112401
:1014E000EF55FE4F6181561306C06081461303C05D
:1014F0006281E61203C001968770E9CFFE2CEE20D0
:1015000009F416C18091D60181608093D60154C040
:101510005E1306C0491304C0E11002C0F80199C06F
:10152000C8010E943807882361F1EE2051F1209113
:10153000D601822F82958F7090E0029774F080918F
:10154000D1019091D20198878F831986BB86AA8694
:101550002C87CE0107960E94BF0686E0F801A1ED18
:10156000B1E001900D928A95E1F70E9463090E9413
:1015700055090AC05E1711F1C8010E943807811190
:101580002CC0C8010E94BF06FF24F394D1C0282FAD
:10159000207F81F77A2DB98AA88A6E2D89890E94C9
:1015A000400781ED91E00E94BF0686E0D6011D92C2
:1015B0008A95E9F70E945509F12CBAC04913DCCF8E
:1015C000E110DACFF8018583C8010E94BF0686E0EA
:1015D000D6011D928A95E9F7ABC0EE2091F22091D9
:1015E000D601822F82958F7090E002970CF4B5CFD0
:1015F0008091D1019091D2019A8389831B82BD820F
:10160000AC822E83CE010196A6CF6217730708F035
:1016100044C0FE2CEE2009F4B4CF5E1330C0491351
:101620002EC02091D60120FD21C0822F82958F707F
:10163000482F50E041155105C9F0F80125834F307E
:10164000510541F08F5F982F9295907F822F8F7078
:10165000892B8583C8010E94BF0686E0F801A1EDB1
:10166000B1E001900D928A95E1F73CC086E0F80167
:10167000A1EDB1E001900D928A95E1F759C0C80142
:101680000E943807811169CF8091D60181608093D3
:10169000D601C8010E94BF064BC07A2DB98AA88A1C
:1016A0006E2D89890E94400786E0D6011D928A9599
:1016B000E9F718C0EE2009F464CFC8010E9438078A
:1016C000F82E882309F45DCF86E0F801A1EDB1E0A2
:1016D00001900D928A95E1F781ED91E00E94B803A7
:1016E0000E9463090E94550923C04D875E878D853E
:1016F0009E850E940609292F22952F70223028F4FA
:101700009F7039F0811105C00BC0243028F49F7000
:1017100049F4805E883020F0C8010E94BF069F2CEB
:10172000F92C06C0D80115969C91907F91F7F8CFBF
:101730008F2D61960FB6F894DEBF0FBECDBFDF913F
:10174000CF911F910F91FF90EF90DF90CF90BF90BE
:10175000AF909F9008951F93CF93DF93CDB7DEB7DF
:101760002C970FB6F894DEBF0FBECDBF4F835887BE
:1017700069877A878B879C87CE0107960E94DB0951
:101780008823D1F09F8188852A853B85232B31F0E2
:101790008F3F31F481E09F3F19F403C081E001C025
:1017A00080E080FD47C04F81588569857A858B85AB
:1017B0009C850E944F073EC086E0FE013796DE0101
:1017C000119601900D928A95E1F7FF81E8856A856F
:1017D0007B856115710531F0EF3F31F481E0FF3F0A
:1017E00019F403C081E001C080E080FD23C0209196
:1017F000A00130E0C90101968770992740919F01AF
:1018000050E084179507F1F1F983EA837D836C83B7
:1018100096E0929FD001939FB00D1124AF55BE4F1B
:10182000FE01319601900D929A95E1F78093A00107
:101830000E94340916E080919F019091A0018917C0
:1018400071F1189FC00111248F559E4F0E94DB0932
:10185000882329F1E0919F011E9FF0011124EF558B
:10186000FE4F4081518162817381848195810E9404
:101870004F0780919F0190E0019687709927809390
:101880009F01D9CF0E9419071092A00110929F01C9
:10189000E1EDF1E086E0DF011D928A95E9F72C96F3
:1018A0000FB6F894DEBF0FBECDBFDF91CF911F9171
:1018B00008958091DF01859585958595089580919E
:1018C000DF01877008959091DF01977081E009F43E
:1018D00080E008958091EA0108959091EA01892BB2
:1018E0008093EA01089580959091EA01892380937D
:1018F000EA0108958093EA0108951092EA0108959B
:101900009091E901892B8093E90108958095909148
:10191000E90189238093E90108951092E90108956E
:101920008091E001089508950C94930C0C94940C0C
:101930009091230292FD08C09091E001981721F048
:101940008093E0010C94960C08958091E001882327
:1019500029F01092E00180E00C94960C0895CF934A
:10196000DF93E0910201F09103018091EA0180830D
:10197000E0910201F091030190818091E901892BAE
:1019800080838091E001882381F0E0910201F09151
:1019900003019081892B8083809102019091030142
:1019A0000E94691881110E94A50CC0910201D0917A
:1019B000030148E050E067ED71E0CE010E94A920EC
:1019C000892B69F088E0FE01A7EDB1E001900D924E
:1019D0008A95E1F7CE01DF91CF910C942418DF9125
:1019E000CF9108950C94930C9091230292FD10C016
:1019F00098E0899F90011124262B2093DF010E94FB
:101A0000D1078091DF018595859585950C94F20C21
:101A10000C94D1071092DF0180E00C94F20C20911D
:101A2000DF01809582238093DF01982F977099F4CE
:101A300030E0482F082E000C550B2417350759F0BD
:101A40009091230292FD07C08595859585950E940A
:101A5000F2070C940A0D08959091230292FB22271D
:101A600020F9281769F080FB92F990932302809166
:101A70002202909123020E94740D82E00C940F0DBB
:101A800008958091230282FB882780F991E08927BD
:101A90000C942C0D81E00C942C0D80E00C942C0DFA
:101AA00080E090E00E94BE2021E0893E9E4F09F038
:101AB00020E0822F089582E090E00C94B62083E02D
:101AC00090E00C94B620CF9384E090E00E94B62082
:101AD000C82F82E290E00E94B6202C2F30E0A901AE
:101AE000582BCA01CF910895CF93C92F682F84E056
:101AF00090E00E94C4206C2F82E290E0CF910C9481
:101B0000C420AB01BC018FE090E00C94D620AB0167
:101B1000BC0183E190E00C94D62060E070E0CB0142
:101B20000C94870D60E070E0CB010E94810D0C9455
:101B30008D0D69EE7EEF80E090E00E94E22060E093
:101B400082E090E00E94C42060E083E090E00E9488
:101B5000C42010929B0110929C0110929D01109242
:101B60009E0160E084E090E00E94C42060E082E298
:101B700090E00E94C42060E085E090E00E94C420D4
:101B800060E086E090E00E94C4206FEF87E090E084
:101B90000E94C42040E050E0BA0188E090E00E943A
:101BA000D62060E08DE090E00E94C42040E050E04C
:101BB000BA0188E190E00E94D62060E087E190E0E1
:101BC0000E94C42040E050E0BA018CE190E00E9405
:101BD000D62060E070E080E290E00E94E22040E0E9
:101BE00050E0BA0188E190E00E94D6200C94920D5A
:101BF0000C94990D682F8EE090E00C94C4200E9404
:101C00005D196093F4017093F5018093F601909350
:101C1000F7016093F0017093F1018093F2019093CA
:101C2000F301089585B7806885BF85B7806885BF53
:101C3000089581E008950C94190E08950C941D0EDA
:101C40000C941D0E0C94200E0C941D0E0C94240E5E
:101C50000C941D0E0E94120E84ED90E10E940B1850
:101C60000E94280E0C94260E0E941E0E0C941D0E2F
:101C70000E94D7100E9452030C940B150E94481921
:101C80000E94AE110E94380E0C94220E8F929F92E9
:101C9000AF92BF92CF92DF92EF92FF920F931F937A
:101CA000CF93DF93CDB7DEB72A970FB6F894DEBF98
:101CB0000FBECDBF0E94C311982E81110E94FF0D4F
:101CC0008BEEA82E81E0B82E00E010E0802E802F51
:101CD0000E94FB10D82EF501C1905F01C826B1F417
:101CE0000F5F1F4F0530110589F78FEF89838A83B6
:101CF0001B820E9451198160782F9D838C834981BA
:101D00005A816B818D810E946E032FC08091F801F2
:101D100081FD0E940111E12CFF24F3948C2D8F2171
:101D2000F1F00E941B0E882399F0EE828F82DF2053
:101D300081E009F480E088870E9451198160782F42
:101D40009A8789874E815F8168858A850E946E03A4
:101D5000F801E551FE4F8081F826F08206C0E39439
:101D6000FF0CF4E0EF12DACFBBCF81E0911001C09D
:101D700080E02A960FB6F894DEBF0FBECDBFDF918C
:101D8000CF911F910F91FF90EF90DF90CF90BF9078
:101D9000AF909F908F9008950E94460E0E94C213AC
:101DA0000C946303CF93DF930E94FD0FEC01811528
:101DB00021E5920708F045C0811530E5930708F04A
:101DC00094C0883E910528F5803E910508F0F8C042
:101DD000883A910570F4853A910508F07CC081300D
:101DE000910509F475C008F4E8C0049708F0E8C04C
:101DF000E4C08F3B910508F0E0C0C85AD0E0CC0F9A
:101E0000DD1FC65BDE4F0990D881C02DCE019464E2
:101E1000D8C0811540E2940758F4811551E0950728
:101E200008F0CEC08D3E910508F4C7C09065C9C0CA
:101E3000C11580E4D80708F4C0C0DF70CE01906AF5
:101E4000C0C0811525E59207A8F4811534E59307F4
:101E500008F095C0811543E5940708F07BC0811513
:101E600052E5950708F061C0D82FCC27CE01816FCD
:101E7000906AA7C0C11589E5D807A0F4C11528E567
:101E8000D20708F082C0C11536E5D30708F095C027
:101E90008C2F0E9491108F7190E0D82FCC27CE010B
:101EA00090628FC0C1154AE5D40708F474C0CE0112
:101EB00090568115904208F080C08D2F8F710E943E
:101EC0009110DD27D0628F71AE01582BCA0179C005
:101ED00081E090E076C0C55AD0E0C858DE4F8881D6
:101EE000C82FD0E0CE0190646CC074E096958795C1
:101EF0007A95E1F7282F23703C2F337081E090E032
:101F000002C0880F991F3A95E2F79C68AC01522BEA
:101F10009A019C2F9F709695969550E2959FE001AF
:101F20001124C9018C2B9D2B4CC08370992721E073
:101F300030E002C0220F331F8A95E2F79C2F96955E
:101F4000969580E2989FE0011124C22BD32BCE01FD
:101F50009C6837C08370992721E030E002C0220FCF
:101F6000331F8A95E2F79C2F9695969540E2949FB1
:101F7000E0011124C22BD32BCE019A6822C0D82FA6
:101F8000CC27CE01846F906A1CC0DC2FCC27CE01F9
:101F9000806F906A16C08C2F8F700E94911094E011
:101FA000D695C7959A95E1F7CF70D0E0DC2FCC2776
:101FB000D0699E01282BC90104C080E090E001C0D7
:101FC000CE01DF91CF910895E72FF0E095E0899F52
:101FD000E00DF11D1124EE0FFF1FEE0FFF1FE60FA6
:101FE000F11DEE0FFF1FE852FF4F85919491089568
:101FF0000E94E40F0E94D20E08958238910569F183
:10200000B0F48133910509F46DC048F4893291052B
:1020100009F463C08A32910509F469C008958533D3
:10202000910509F455C089339105B9F00895833EAF
:10203000910569F138F4803E9105B1F0823E910539
:1020400009F10895863E9105A9F1873E9105B9F100
:10205000843E910509F064C023C02091220220FD36
:102060004FC021FD4DC008958091220280FD44C0E3
:102070008091230280FF44C08091220284FD42C0EF
:1020800083EE4DC08091220282FF38C0F5CF80914F
:10209000220282FD33C08091230280FD31C0ECCF4B
:1020A0008091230281FF32C08091220284FD2AC0E8
:1020B00087EE35C08091220283FF26C0F5CF809144
:1020C000220283FD21C08091230281FD1FC0ECCF3D
:1020D0008091220285FD1CC01DC08091220285FDD9
:1020E00019C016C08091220286FD16C017C08091CB
:1020F000220286FD13C010C089E311C082EE0FC01A
:1021000080EE0DC080E00BC086EE09C084EE07C0F3
:1021100089E205C085E303C08AE201C081E390E063
:1021200008959091220292FF0DC0282F2871283027
:1021300019F4877F846006C0282F2471243011F49D
:102140008B7F886093FF0DC0282F2871283119F4E8
:10215000877E846106C0282F2471243111F48B7E80
:1021600088612091230220FF0DC0382F387138304C
:1021700019F4877F816006C0382F3171313011F436
:102180008E7F886021FF0DC0282F2871283119F417
:10219000877E816106C0282F2171213111F48E7E46
:1021A000886194FD877E089580E0089508950E94D7
:1021B000500D811102C00E94F80D0E945B0D8093AA
:1021C000F8010E94630D90932302809322020E94E3
:1021D000D6100E945F0D682F70E080E090E00E94B2
:1021E0007107609197017091980180919901909188
:1021F0009A010C94A907E82FF0E0E75DFD4F80817C
:102200000895089580EA8A95F1F7089500C0089529
:102210000C94021108950C940A110C940B110C9457
:102220000A110C940F11F894E82FE295EF70F0E08A
:1022300031A1282F2F7081E090E001C0880F2A95EE
:10224000EAF7982F9095932391A392A1892B82A3CB
:10225000789408950F931F93CF93DF93CFE7D1E046
:1022600089918F3F11F00E94131181E0C438D80783
:10227000B9F7CBE7D1E00FE711E089918F3F11F07B
:102280000E9413110C171D07C1F7DF91CF911F9109
:102290000F910895CF92DF92EF92FF920F931F93C9
:1022A000CF93DF938C01C62FD0E0CE0181589E4F93
:1022B0007C01FC0190819F3F09F447C0D62EF89421
:1022C000E92FE295EF70F0E081A19F7021E030E00E
:1022D00001C0220F9A95EAF7822B81A382A1209553
:1022E000282322A378940E940611EBE7F1E04FE740
:1022F00051E031E0C12C21912F3F89F0A22FA2950E
:10230000AF70B0E090968C9190E02F7002C09595E0
:1023100087952A95E2F780FD02C0832F01C080E0F7
:10232000C82A330F4E175F0731F7F70180818F3FBF
:1023300011F00E94131161E0C11001C060E08D2D09
:102340000E940811C00FD11FC882DF91CF911F9149
:102350000F91FF90EF90DF90CF9008950E942A1187
:1023600085E0E9E2F2E0DF01982F1D929A95E9F706
:10237000E4E2F2E0DF011D928A95E9F785E00E9430
:102380000A120C946602FF920F931F93CF93DF9370
:1023900000D000D01F92CDB7DEB78E010F5F1F4F68
:1023A00085E0F80111928A95E9F7F12C6F2DC801AB
:1023B0000E944A11F394F5E0FF12F8CF45E050E097
:1023C000B80184E292E00E94A920FF24F3940097D0
:1023D00009F4F12C892B41F085E0F801A4E2B2E088
:1023E00001900D928A95E1F72F2D45E069E272E0A8
:1023F00084E292E00E940B120E9468028F2D0F90DF
:102400000F900F900F900F90DF91CF911F910F9130
:10241000FF9008950895FF920F931F93CF93DF933A
:102420008C01F62ED72FC42F222349F081E0809310
:10243000FB010E9451199093FA018093F901809158
:10244000FB018823C1F08091F9019091FA010E946B
:102450006919059780F0EF2DFD2FD8014C2F50E022
:10246000CD01801B910B841795071CF48D918193EE
:10247000F7CF1092FB01DF91CF911F910F91FF9049
:1024800008950E94411B0E943E0E0C944D1B0E9419
:10249000511B0E94CC0E0C946B1B0E94EF180E94E3
:1024A000281B0E942A0E0E9441120E9447120E947D
:1024B000340EFBCF8091020280FF06C060910901BB
:1024C00070E0660F771F26C081FF04C0609109018C
:1024D00084E005C082FF07C06091090188E0689F21
:1024E000B001112417C0909101029923D1F060919D
:1024F0000801961788F72091090188E0289F90012C
:102500001124929FA001939F500D112470E0CA01E5
:102510000E947B206038710540F46115710519F443
:1025200006C068E070E0862F08958FE7089581E087
:1025300008958091020280FF08C06091050170E05B
:10254000759567957595679521C081FF06C0609167
:10255000050170E07595679519C082FF04C0609110
:10256000050170E010C090910002992399F06091EC
:1025700004019617A0F780910501899FC0011124DD
:1025800070E00E947B206038710540F46115710590
:1025900019F406C061E070E0862F08958FE7089572
:1025A00081E008958D3E21F40E945A12819504C065
:1025B0008E3E29F40E945A128093060208958F3E9F
:1025C00021F40E945A12819504C0803F29F40E9490
:1025D0005A12809305020895893F19F40E949912B6
:1025E00005C08A3F31F40E949912819580930702B9
:1025F00008958B3F21F40E949912819504C08C3F6D
:1026000029F40E9499128093080208959FE0980F80
:10261000983078F421E030E0A90102C0440F551F42
:102620009A95E2F7CA0190910402892B80930402E3
:1026300008958D3F21F48091020281600BC08E3F8E
:1026400021F480910202826005C08F3F29F48091BD
:10265000020284608093020208958D3E39F49091C5
:10266000060297FF35C01092060259C08E3E29F42B
:10267000909106021916BCF32BC0909105028F3E73
:1026800029F497FF25C01092050249C0803F19F434
:102690001916CCF31DC090910702893F29F4191631
:1026A000BCF4109207023BC08A3F19F497FF10C098
:1026B000F8CF8B3F39F49091080297FF09C0109230
:1026C00008022DC08C3F21F4909108021916BCF32A
:1026D0009FE0980F983080F421E030E0A90102C01B
:1026E000440F551F9A95E2F7CA0180959091040214
:1026F00089238093040213C08D3F21F4809102024C
:102700008E7F0BC08E3F21F4809102028D7F05C029
:102710008F3F29F4809102028B7F80930202809187
:102720000502811106C080910602811102C010923B
:10273000010280910702811106C080910802811177
:1027400002C01092000208950E94511920910502C2
:10275000211104C020910602222321F09093FF0151
:102760008093FE0120910702211104C020910802EC
:10277000222321F09093FD018093FC0183E092E0FD
:102780000C942F18EF92FF920F931F93CF93DF9328
:1027900000D000D000D0CDB7DEB786E0E3E0F2E0B5
:1027A000DE01119601900D928A95E1F7E090050205
:1027B000F0900602009107021091080210920502A3
:1027C000109206021092070210920802E11003C054
:1027D000FF2009F45DC08091FE019091FF010E94ED
:1027E0006919AC0190910102992339F020910A01F5
:1027F00030E02417350758F04BC020910B018AE0D8
:10280000289F900111242417350718F041C09F3FDD
:1028100019F09F5F90930102EE2061F00E945A121E
:102820001E1414F09FEF01C091E0989F902D112489
:1028300090930502FF2061F00E945A121F1414F0B9
:102840009FEF01C091E0989F902D11249093060274
:10285000309105023323E1F0209106022223C1F0DA
:1028600045EB3403C0011124992319F0909305021C
:1028700003C081E08093050235EB2303C0011124DE
:10288000992319F09093060203C081E08093060219
:10289000011103C0112309F45DC08091FC019091E6
:1028A000FD010E946919AC0190910002992339F051
:1028B0002091060130E02417350758F04BC02091D5
:1028C00007018AE0289F900111242417350718F08A
:1028D00041C09F3F19F09F5F90930002002361F079
:1028E0000E949912101614F09FEF01C091E0989F7A
:1028F000902D112490930702112361F00E949912E8
:10290000111614F09FEF01C091E0989F902D1124B3
:1029100090930802309107023323E1F020910802DE
:102920002223C1F045EB3403C0011124992319F08F
:102930009093070203C081E08093070235EB2303E5
:10294000C0011124992319F09093080203C081E07B
:10295000809308028091050281110BC080910602CC
:10296000811107C080910702811103C08091080284
:1029700081110E94A413EB82FC820D831E8386E0EA
:10298000FE013196A3E0B2E001900D928A95E1F745
:1029900026960FB6F894DEBF0FBECDBFDF91CF9164
:1029A0001F910F91FF90EF900895E3E0F2E086E031
:1029B000DF011D928A95E9F7109201021092000240
:1029C000109202020895CF93DF9397FF0DC0FB0191
:1029D0002281222349F0EC010E942115CE019F772C
:1029E0000E9494150E946E1581E0DF91CF910895A9
:1029F00090912F02923069F48A3040F490E0099669
:102A00006AE070E00E947B20875A01C086500C94D7
:102A10005F040C9441038CE090E00E94B62090E0AB
:102A2000A0E0B0E080932F0290933002A093310297
:102A3000B0933202089560912F028CE090E00C94E4
:102A4000C4200E94211886958170809334020E94D0
:102A50002118817080932E0280912F02813039F4E9
:102A600080913402882319F089E30E945F040E9458
:102A70006A0C809333020E947D0C80912F0281307A
:102A800071F048F0823081F0843009F586EE0E94C2
:102A90005F0488E11AC082EE0E94BE0318C088E17C
:102AA00093E00E94000213C080912E02811103C0A6
:102AB00083E50E945F0482EE0E94BE038FE39CE9DF
:102AC0000197F1F700C0000087E50E945F048FE3E3
:102AD0009CE90197F1F700C00000089580912F0252
:102AE000813059F030F0823089F08430C9F488E2C6
:102AF00015C082EE0E94140413C08CE20E945F0491
:102B000080913402882361F089E308C082EE0E943C
:102B1000140480912E02811103C083E50E945F049A
:102B2000809133020C947A0C0F931F93CF93DF9311
:102B30008C01CCE0D0E0C8010C2E02C096958795A0
:102B40000A94E2F78F700E94F8142497CC3F8FEF1D
:102B5000D80789F7DF91CF911F910F9108950F93B7
:102B60001F93CF93DF93EC018B01FB0182818823BC
:102B700061F00E946A0CCE01825E9C458530910511
:102B800020F480932F020E941B15B801CE01DF9123
:102B9000CF911F910F910C94E314CF93DF93EC012D
:102BA000FB018281882309F43CC1C430FDE5DF07C5
:102BB00060F4CB3F9CE5D90788F49E0122503C4548
:102BC0002431310508F02EC109C0C236EDE5DE071B
:102BD00029F0C63AFDE5DF0709F024C10E94630D24
:102BE0009093230280932202C1318CE5D80709F427
:102BF000C6C008F042C0C930ECE5DE0709F49BC04E
:102C000000F5C5308CE5D80709F485C078F4C330E9
:102C1000ECE5DE0709F478C008F07AC0C230DC4584
:102C200009F0F5C0809122028160EFC0C7309CE5B9
:102C3000D90709F478C008F07AC080912202806137
:102C4000E4C0CD30FCE5DF0709F487C058F4CB3091
:102C50009CE5D90709F479C008F07BC08091220275
:102C600088606FC0CF30FCE5DF0709F480C008F052
:102C700082C080912202877FC8C0CE3F9CE5D907E1
:102C800009F471C000F5C531FCE5DF0709F485C022
:102C900068F4C3319CE5D90709F475C008F095C004
:102CA0000E941907809122028F77AFC0CC3FFCE5CC
:102CB000DF07A9F108F054C0CB3FDC4509F0A7C0FD
:102CC0008091230240C0C230EDE5DE0709F489C0DF
:102CD00058F4C1158DE5D80709F45AC008F069C049
:102CE0008091230282602FC0C236EDE5DE0709F431
:102CF0007CC0C63AFDE5DF0709F481C0C330DD457D
:102D000009F085C080E06EC08091220282607DC0A3
:102D10008091220216C080912202886076C0809144
:102D2000230282604FC08091220280626EC0809137
:102D3000220280646AC00E94190780912202806882
:102D400064C0846062C081603DC0809122028E7F39
:102D50005CC0809122028D7F58C08091220216C0F3
:102D60008091230218C0809123028D7F2BC0809117
:102D700022028F7E4AC0809122028F7D46C08091C0
:102D800022028F7B42C080912202877F8B7F3DC0D1
:102D9000809123028D7F8E7F15C08091220282FB5D
:102DA000222720F991E0922790FB82F990FB83F98A
:102DB0002CC080912302982F909591708E7F892B43
:102DC00090FB81F98093230222C00E941907809111
:102DD000220287FB222720F991E0922790FB87F9B6
:102DE00014C081E00E94FA0D12C08091220284FB7F
:102DF000222720F991E0922790FB84F906C0809168
:102E00002202982F909590FB80F980932202809166
:102E10002202909123020E94740D0E94190780E003
:102E200001C081E0DF91CF910895CF93DF93863188
:102E30009C4541F5EB010E946A0C982F8A812091F4
:102E4000020130910301882379F09A7A81E009F434
:102E500080E080930902911102C069E201C065E33C
:102E6000C9010E94AB180AC080910902811102C0F9
:102E700069E201C065E3C9010E94AD180E94AF0C70
:102E800080E001C081E0DF91CF9108950F931F93FF
:102E9000CF93DF93C42FD22FFC0182818823C9F006
:102EA00040930C020E94511990930B0280930A02E6
:102EB00080E28C0F883008F057C0C77081E001C0F5
:102EC000880FCA95EAF7DF91CF911F910F910C946B
:102ED000680480910C02481330C080910A029091DE
:102EE0000B020E946919883C910538F510E21D0F0C
:102EF000CD17B9F080E28C0F883040F4C77081E0C4
:102F000001C0880FCA95EAF70E946F04183028F5AF
:102F100081E09D2F977001C0880F9A95EAF70E9473
:102F20006804802F0E945F041830F0F4D77081E0AD
:102F300001C0880FDA95EAF70AC080E28C0F88306A
:102F400098F4C77081E001C0880FCA95EAF7DF9155
:102F5000CF911F910F910C946F04802FDF91CF912F
:102F60001F910F910C945F04DF91CF911F910F91EE
:102F700008950F939C01CB01243F4CE5340731F1B8
:102F800088F4293DFCE53F07D9F02A3D4CE534079C
:102F900079F1283D3C45A9F506E221EE41EE68EDC8
:102FA0007CE52BC0263FFCE53F07E1F0A8F0273F7A
:102FB0003C4539F507E225EE46EE67EF7CE51DC09E
:102FC00007E225EE45EE69ED7CE517C006E221EE4D
:102FD00040EE64EF7CE511C007E225EE44EE65EFBC
:102FE0007CE50BC006E221EE42EE66EF7CE505C013
:102FF00008E221E045EE6AED7CE50E94461780E09C
:1030000008C0FC018281882319F010920C0201C0D3
:1030100081E00F9108959093850180938401089534
:1030200090931202809311020895E0911102F091A1
:103030001202309721F00190F081E02D099480E098
:1030400008950E9415180895E0911102F09112025E
:10305000309721F00280F381E02D09940895E091EA
:103060001102F0911202309739F022E0DC012C932A
:103070000480F581E02D0994089520910F0230918C
:1030800010022817390771F09093100280930F02F5
:10309000E0911102F0911202309721F00680F78141
:1030A000E02D0994089520910D0230910E02281709
:1030B000390771F090930E0280930D02E091110296
:1030C000F0911202309721F00084F185E02D0994EF
:1030D0000895FC01329697E080E0915029F021910B
:1030E0002223D9F38F5FF9CF0895662349F0FC01BD
:1030F000329608962191621729F0E817F907D1F75F
:1031000080E0089581E008959C01FC0132969FEFD4
:1031100080E04191461789F09F3F19F4411101C0A9
:10312000982F8F5F8630A9F79F3F39F0F901E90F9B
:10313000F11D97FDFA956283089508959C012A5F19
:103140003F4FFC014281461301C012820196821753
:103150009307B9F708950C9484180C949E1802965E
:1031600026E0FC0111922A95E9F7089508950C9440
:10317000B61883E0809313020C94B718811102C033
:1031800081E001C082E0809313020C94B7180C9484
:10319000BE1881E0809313020C94B7180C94C918E0
:1031A00008950C94D0180C94D1180C94D0180C9449
:1031B000D0180C94D018CF930E94D7180E94C31136
:1031C0000E94D518C0E08C2F0E94FB10811104C012
:1031D000CF5FC530C1F701C081E0CF910895089558
:1031E0001F920F920FB60F9211248F939F93AF935C
:1031F000BF9380911402811113C080913502909188
:103200003602A0913702B09138024196A11DB11D3E
:103210008093350290933602A0933702B093380220
:10322000BF91AF919F918F910F900FBE0F901F9004
:10323000189580913D02843031F10E94D3021092A2
:10324000140220E488E190E00FB6F894A8958093EA
:1032500060000FBE2093600083B7817F846083BFCE
:1032600083B7816083BF7894889583B78E7F83BF4F
:103270000FB6F894A89580916000886180936000F3
:10328000109260000FBE08950E9419070C94D70297
:1032900082E084BD93E095BD9AEF97BD80936E0068
:1032A00008952FB7F8948091350290913602A0913D
:1032B0003702B09138022FBF08952FB7F89460916C
:1032C00035027091360280913702909138022FBFFB
:1032D00008959C014FB7F894809135029091360281
:1032E000A0913702B09138024FBF821B930B089513
:1032F00078941F920F920FB60F9211248F939F9381
:10330000AF93BF938091350290913602A09137021E
:10331000B09138020196A11DB11D809335029093A2
:103320003602A0933702B0933802BF91AF919F91BC
:103330008F910F900FBE0F901F90189587E797E71A
:1033400090930108809300089AE088E10FB6F89402
:10335000A895809360000FBE90936000FFCF80918E
:1033600020020895089522E02093E9002FEF309184
:10337000E800215035FD06C035ED3A95F1F7000023
:103380002111F5CF2091E80025FF0BC040E050E06F
:1033900066E070E00E94DD1B8091E8008E778093EC
:1033A000E8000895CF93DF9321E02093E9002FEF09
:1033B0003091E800215035FD06C035ED3A95F1F722
:1033C00000002111F5CF2091E80025FF14C0EC0189
:1033D00040E050E068E070E00E94DD1B8091E80072
:1033E0008E778093E80088E0FE01A8E1B2E00190CA
:1033F0000D928A95E1F7DF91CF91089580931502A0
:10340000709317026093160280913D02843001F59B
:1034100082E08093E9008FEF9091E800815095FD64
:1034200006C095ED9A95F1F700008111F5CF8091D6
:10343000E80085FF0DC040E050E063E070E085E10A
:1034400092E00E94DD1B8091E8008E778093E80077
:103450000895BC0184E00C94FE19BC0183E00C9437
:10346000FE1980913C02811109C00E946E1D0E94CC
:10347000CB1D8091E20084608093E2000895109259
:103480003C0208950C94CE186091390281E06111DC
:1034900001C080E00C94B91890913D0281E0943015
:1034A00009F080E0609139020C94BE1842E061ECB2
:1034B00081E00E94E71C42E261EC82E00E94E71C8E
:1034C00090913D0281E0943009F080E060913902F2
:1034D0000C94C71880913F02833009F461C030F426
:1034E000813071F0823009F49AC008958A3009F46D
:1034F00086C08B3009F46CC0893009F0A8C020C0A8
:1035000080913E02813A09F0A2C08091E800877F55
:103510008093E8008091420290914302892B21F42C
:1035200068E088E192E003C060E080E090E070E055
:103530000E94281C8091E8008B778093E800089512
:1035400080913E02813209F082C0809142029091C6
:103550004302029708F07BC08091E800877F809348
:10356000E8008091E80082FD05C080913D02811154
:10357000F8CF6DC02091F3008091F20090E0922B83
:10358000029731F48091F100813011F0863021F4FE
:103590008091F100809320028091E8008B7753C0E6
:1035A00080913E02813A09F052C08091420290918E
:1035B0004302892B09F04BC08091E800877F8093FC
:1035C000E8008091E80080FFFCCF8091180136C0B0
:1035D00080913E028132D9F580914202909143025E
:1035E000892BA9F58091E800877F8093E8000E94ED
:1035F0001C1D80914002809318010C941907809142
:103600003E02813221F58091E800877F8093E800B7
:103610000E941C1D80914102809321020895809197
:103620003E02813AA1F48091E800877F8093E80010
:103630008091E80080FFFCCF809121028093F1000F
:103640008091E8008E778093E8000C941C1D08950B
:1036500084B7877F84BF0FB6F894A89580916000E7
:10366000886180936000109260000FBE90E080E857
:103670000FB6F89480936100909361000FBE0C9494
:10368000C9180E946E1D0E94CB1DE2EEF0E0808101
:103690008460808378940C9460208CE091E00C949A
:1036A000101880913D028530A9F480913D0285304B
:1036B00079F40E94191980913B028823B1F30E948A
:1036C000DB18882391F30E94C71B0E941907EDCFD6
:1036D0000C944419089508950C946E1B292F3327D8
:1036E00023303105C9F060F42130310581F02230FA
:1036F000310509F044C08BE390E028ED31E043C090
:1037000021323105E1F02232310549F138C082E140
:1037100090E023E132E037C099278130910549F0EC
:1037200028F0029761F5E0EBF1E005C0E4EDF1E08F
:1037300002C0E4ECF1E0849190E09F0124C06115A7
:10374000710541F061307105D1F489E090E023E02A
:1037500032E019C089E090E02AEE31E014C0611532
:10376000710541F06130710551F48BE790E025E27D
:1037700032E009C080E490E020EA32E004C080E05A
:1037800090E020E030E0FA0131832083089580E169
:1037900089BD82E189BD09B400FEFDCF8091D800CA
:1037A0008F7D8093D8008091E00082608093E0005C
:1037B0008091E00081FDFCCF0895CF92DF92EF92DF
:1037C000FF920F931F93CF93DF93EC018B017A014C
:1037D0000E943B1D811133C0E114F10439F0F7015F
:1037E00080819181081B190BC80FD91FC12CD12CC6
:1037F0000115110519F18091E80085FD16C0809131
:10380000E8008E778093E800E114F10449F0F701B5
:1038100080819181C80ED91ED182C08285E00FC0FF
:103820000E943B1D882321F30AC089918093F100F7
:1038300001501109FFEFCF1ADF0ADACF80E0DF91E4
:10384000CF911F910F91FF90EF90DF90CF9008954F
:1038500020914402309145022617370748F0611540
:10386000710539F42091E8002E772093E80001C01B
:10387000B901FC0120E06115710579F180913D02EB
:103880008823F1F18530F1F18091E80083FD3CC09F
:103890008091E80082FD2EC08091E80080FFEBCF90
:1038A0002091F3008091F20090E0922B6115710558
:1038B00051F08830910538F421912093F100615046
:1038C00071090196F3CF21E0089709F020E080917B
:1038D000E8008E778093E800CECF2111CFCF0AC0C9
:1038E00080913D02882361F0853061F08091E8008D
:1038F00083FD0AC08091E80082FFF2CF80E0089546
:1039000082E0089583E0089581E0089520914402C3
:10391000309145022617370748F06115710539F4D3
:103920002091E8002E772093E80001C0B901FC0146
:1039300020E06115710591F180913D02882309F421
:1039400040C0853009F43FC08091E80083FD3DC050
:103950008091E80082FD2FC08091E80080FFE9CFD0
:103960002091F3008091F20090E0922B6115710597
:1039700059F08830910540F424912093F10031965C
:10398000615071090196F2CF21E0089709F020E01B
:103990008091E8008E778093E800CBCF2111CCCFC7
:1039A0000AC080913D02882361F0853061F08091EA
:1039B000E80083FD0AC08091E80082FFF2CF80E03A
:1039C000089582E0089583E0089581E00895982F96
:1039D000973068F59093E900981739F07091EC00F2
:1039E0002091ED005091F00003C0242F762F50E07D
:1039F00021FD02C09F5FECCF3091EB003E7F309302
:103A0000EB003091ED003D7F3093ED003091EB0005
:103A100031603093EB007093EC002093ED005093F5
:103A2000F0002091EE0027FDE5CF80E008958F7033
:103A30008093E90081E0089580913E0287FF11C0E4
:103A40008091E80082FD05C080913D028111F8CF90
:103A500011C08091E8008B770BC080913D028823D4
:103A600049F08091E80080FFF8CF8091E8008E77E0
:103A70008093E80008952091E4003091E50095E6F8
:103A80004091EC00842F817040FF23C08091E800BA
:103A900080FD1DC080913D02882399F0853099F00A
:103AA0008091EB0085FD11C04091E4005091E5004C
:103AB0002417350729F3915011F09A01E1CF84E0E2
:103AC000089582E0089583E0089581E0089580E0FC
:103AD00008954091E80042FFDDCF08950E94DC1D6B
:103AE0000E94E41DE0EEF0E0808181608083E8EDDB
:103AF000F0E080818F77808319BCA7EDB0E08C91D6
:103B00008E7F8C9380818F7E808310923C020895FB
:103B10000F931F93CF93DF930E94DC1D0E94E41D3F
:103B2000C8EDD0E088818F7788838881806888831A
:103B300088818F7D888319BC10923D0210923902D2
:103B400010923B0210923A0200EE10E0F8018081E0
:103B50008B7F808388818160888342E060E080E0A1
:103B60000E94E71CE1EEF0E080818E7F8083E2EE30
:103B7000F0E0808181608083808188608083F801AB
:103B800080818E7F8083888180618883DF91CF915F
:103B90001F910F910895E8EDF0E080818F7E808382
:103BA000E7EDF0E080818160808384E082BF81E086
:103BB00080933C020C94881DE8EDF0E080818E7FBC
:103BC00080831092E20008951092DA001092E100D2
:103BD00008951F920F920FB60F9211242F933F93C7
:103BE0004F935F936F937F938F939F93AF93BF9305
:103BF000EF93FF938091E10082FF0BC08091E20080
:103C000082FF07C08091E1008B7F8093E1000E94DA
:103C10005F208091DA0080FF1FC08091D80080FF74
:103C20001BC08091DA008E7F8093DA008091D900EA
:103C300080FF0DC080E189BD82E189BD09B400FE2D
:103C4000FDCF81E080933D020E94311A05C019BC6E
:103C500010923D020E943F1A8091E10080FF19C03E
:103C60008091E20080FF15C08091E2008E7F8093FA
:103C7000E2008091E20080618093E2008091D800B0
:103C800080628093D80019BC85E080933D020E9439
:103C9000441A8091E10084FF30C08091E20084FFEB
:103CA0002CC080E189BD82E189BD09B400FEFDCF51
:103CB0008091D8008F7D8093D8008091E1008F7E25
:103CC0008093E1008091E2008F7E8093E2008091FA
:103CD000E20081608093E20080913902882311F034
:103CE00084E007C08091E30087FD02C081E001C04D
:103CF00083E080933D020E944C1A8091E10083FF93
:103D000029C08091E20083FF25C08091E100877F78
:103D10008093E10082E080933D021092390280910D
:103D2000E1008E7F8093E1008091E2008E7F80939E
:103D3000E2008091E20080618093E20042E060E076
:103D400080E00E94E71C8091F00088608093F00082
:103D50000E94421AFF91EF91BF91AF919F918F9175
:103D60007F916F915F914F913F912F910F900FBE77
:103D70000F901F9018951F920F920FB60F9211245B
:103D80002F933F934F935F936F937F938F939F9363
:103D9000AF93BF93CF93DF93EF93FF93C091E9006D
:103DA000CF708091EC00D82FD17080FDD0E81092B8
:103DB000E9008091F000877F8093F00078940E9462
:103DC000FF1E1092E9008091F00088608093F0005F
:103DD000CD2BCF70C093E900FF91EF91DF91CF9190
:103DE000BF91AF919F918F917F916F915F914F9113
:103DF0003F912F910F900FBE0F901F9018951F931A
:103E0000CF93DF93CDB7DEB7AA970FB6F894DEBF96
:103E10000FBECDBFEEE3F2E08091F100819322E08E
:103E2000E634F207C9F70E946A1A8091E80083FF1E
:103E30002EC180913E0290913F02492F50E04A30BE
:103E4000510508F024C1FA01EE59FF4F0C948F2060
:103E5000803821F0823809F01AC108C080913A02F6
:103E600090913B02992389F082600FC080914202B9
:103E70008F70873008F00BC18093E9008091EB00D0
:103E800085FB882780F91092E9009091E800977FE0
:103E90009093E8008093F1001092F100D1C0282F98
:103EA0002D7F09F0F4C0882319F0823061F0EFC053
:103EB00080914002813009F0EAC0933009F080E03F
:103EC00080933B022EC08091400281112AC08091D4
:103ED00042028F702FEF280F263008F0D8C0809351
:103EE000E9002091EB0020FF1CC0933021F4809169
:103EF000EB00806214C09091EB0090619093EB0016
:103F000021E030E0A90102C0440F551F8A95E2F775
:103F10004093EA001092EA008091EB008860809361
:103F2000EB001092E9008091E800877F8093E80021
:103F30000E941C1DACC08111AAC0109140021F77C5
:103F40008091E3008078812B8093E3008091E800EA
:103F5000877F8093E8000E941C1D8091E80080FF0D
:103F6000FCCF8091E30080688093E300111102C0D0
:103F700082E001C083E080933D0289C08058823096
:103F800008F085C080914002909141028C3D53E041
:103F9000950779F583E08A838AE289834FB7F8949D
:103FA000DE01139620E03EE051E2E32FF0E0509373
:103FB0005700E49120FF03C0E295EF703F5FEF7080
:103FC0008E2F90E0EA3010F0C79601C0C0968D9316
:103FD0009D932F5F243149F74FBF8091E800877F81
:103FE0008093E8006AE270E0CE0101960E94281CEE
:103FF00016C06091420270914302AE014F5F5F4F65
:104000000E946C1BBC01892B09F441C09091E8000F
:10401000977F9093E80089819A810E94861C809105
:10402000E8008B778093E80032C0803881F580917A
:10403000E800877F8093E800809139028093F10047
:104040008091E8008E7772CF811121C0809140026B
:104050009091410299270297D4F48091E800877FDC
:104060008093E80080914002809339020E941C1DD9
:1040700080913902811106C08091E30087FD02C062
:1040800081E001C084E080933D020E94561A809135
:10409000E80083FF0AC08091E800877F8093E800F2
:1040A0008091EB0080628093EB00AA960FB6F894A3
:1040B000DEBF0FBECDBFDF91CF911F910895089550
:1040C000CF9380913D028823A1F0C091E900CF7089
:1040D0009091EC00892F817090FD80E8C82B1092A0
:1040E000E9008091E80083FD0E94FF1ECF70C0931D
:1040F000E900CF91089597FB072E16F4009407D09E
:1041000077FD09D00E94952007FC05D03EF49095DC
:1041100081959F4F0895709561957F4F0895EE0F9B
:10412000FF1F0590F491E02D0994AA1BBB1B51E1E0
:1041300007C0AA1FBB1FA617B70710F0A61BB70B17
:10414000881F991F5A95A9F780959095BC01CD01BC
:104150000895FB01DC0104C08D910190801921F4C8
:1041600041505040C8F7881B990B0895F999FECF2C
:1041700092BD81BDF89A992780B50895A8E1B0E075
:1041800042E050E00C94EA20262FF999FECF92BD30
:1041900081BDF89A019700B4021639F01FBA20BD0C
:1041A0000FB6F894FA9AF99A0FBE08950396272F3E
:1041B0000E94C5200E94C420252F0E94C520242FC4
:1041C0000C94C5200196272F0E94C5200C94C42072
:1041D000DC01CB01FC01F999FECF06C0F2BDE1BDC7
:1041E000F89A319600B40D9241505040B8F70895B6
:0441F000F894FFCF71
:1041F400C800E101280850011E0A1401AF19D219A0
:10420400B3192D1A291AB21901E200E900EA00B51E
:1042140000B600B700CD008301CC008A019201945E
:10422400012102230224022502260227022A02B3C4
:1042340000B4006F007000818283E200E900EA00AC
:10424400B500B600B700CD008301CC008A0192010D
:1042540094012102230224022502260227022A02B3
:10426400B300B4006F007000818283919094326631
:0442740097C6343580
:00000001FF
